:10000000830100308A008A28F70003088301BC00BE
:100010000408BD000A08BE008A010B1D53280B11FD
:10002000831203132708031D28282208031DA20397
:10003000280803192028A01E1F288614202806142B
:10004000290803192828201F27288615282806157F
:1000500028082702031C2E28FC30860529082702C1
:10006000031C3428F330860503302702031C402884
:10007000861A8610061A0610861B8611061B0611A4
:10008000A70AA7138316981C532883122B082A0645
:10009000031954282B08B03E8400831300089900EC
:1000A000AB0A1F30AB05831203130C1D6B28171C02
:1000B0005F281508AE001608AF00043069282E0826
:1000C0001502AC002F08031C2F0A1602AD002014E5
:1000D000053097000C110D1C81281D1C75281B086C
:1000E000B2001C08B30004307F2832081B02B000A5
:1000F0003308031C330A1C02B100A01405309D0014
:100100000D103D0884003E088A003C088300F70E6D
:10011000770E09002030840021309D20213084009A
:100120003C309D20A0308400D0309D2083010A12F5
:100130008A114C2F04068001840A0406031D9A28A4
:100140000034BF00C01BAB2840088A003F08BF0A2C
:100150000319C00A82008313401883173F08BF0A9F
:1001600084000008080082073034313432343334DC
:100170003434353436343734383439344134423415
:08018000433444344534463495
:100AE40083120313B400B40A340884008313073058
:100AF40080053408840083130008350784008313B9
:100B040034088000B601B701B50135083507840003
:100B140083130008F000F101F01BF103B60703187A
:100B2400B70A7108B707B50A08303502031C872DC8
:100B34000830F200F3013608F0003708F1000A1219
:100B44008A11B4277408B6007508B700360808007F
:100B540083120313B4002A0AB5001F30B505350803
:100B64002B06031900342A08B03E8400831334088A
:100B740080003508AA00013483120313B400003046
:100B84008A0083120313340E0F39B3200A128A1118
:100B9400AA2500380319C12D00308A0034080F3902
:100BA400B3200A128A11AA250038031D0800CE2D8D
:100BB400EA2D3508C00034080A128A11A1200A124D
:100BC4008A11AA2500380319EA2DB40A0319B50AB3
:100BD400831203133508C00034080A128A11A120B5
:100BE4000A128A11003803190800DB2D831203133B
:0C0BF40024082302B800B901031CB90357
:100C0000A31BB903A41BB90A2408F000F101F01BCF
:100C1000F1032308803E0318F103803EF007031818
:100C2000F10AF009F109F00A0319F10A7008BA0093
:100C30007108BB00B91F232EB809B909B80A0319F6
:100C4000B90AA016242EA0123908803AF00080308C
:100C50007002803003193802031C312E7F30B80037
:100C6000B9013808B7000A303702031CB70137084A
:100C7000A800BB1F422EBA09BB09BA0A0319BB0A56
:100C80002017432E20133B08803AF000803070027A
:100C9000803003193A02031C502E7F30BA00BB018A
:100CA0003A08B7000A303702031CB7013708A90019
:100CB000080083120313B800B701B8080319672EA0
:100CC0003818B70A0310B80CB808031D602E37088F
:100CD000080083120313B700A60A0730A6052608EA
:100CE000A83E8400831337088000B901BA01B80117
:100CF0003808A83E840083130008F000F101F01BBF
:100D0000F103B9070318BA0A7108BA07B80A08301C
:100D10003802031C782E0830F200F3013908F00085
:100D20003A08F1000A128A11B4277408B90075084C
:100D3000BA003908080083120313B700A50A073068
:100D4000A5052508A03E8400831337088000B9015B
:100D5000BA01B8013808A03E840083130008F000EF
:100D6000F101F01BF103B9070318BA0A7108BA07B9
:100D7000B80A08303802031CAA2E0830F200F3012A
:100D80003908F0003A08F1000A128A11B4277408F1
:100D9000B9007508BA00390808001230F200F301F2
:100DA000831203133808F1003708F0000A128A1181
:100DB000C9270A128A117408BA007508BB00673087
:100DC000BA070318BB0AFE30BB073B08803AF000A5
:100DD00080307002803003193A02031CF22E7F30FB
:100DE000BA00BB013B08803AF0007F3070028130CE
:100DF00003193A020318002F8130BA00FF30BB00FC
:100E00003A08B90008002A30831203133802F93077
:100E100003193702031C0E2F031008000F3038028D
:100E2000A0300319370208008312031385018601DD
:100E30008701C63083168700F0308600C0308500F9
:100E400006309F0083129F01053097009D000130FE
:100E500090001F3083169900903083129800A230C2
:100E600083169800831281016400DC3083168100B0
:100E700083128101FF30831692007E30831292002C
:100E80008C10FF30A100043083168C0001308D00DF
:100E9000E0308B00831208001427201C6A2F2010DA
:100EA0002C08B5002D08B600A0150310A10D3508BB
:100EB000B7003608B8000327031C692F3508B700B0
:100EC0003608B800CD26A3009B260A128A11A3007B
:100ED0006A2F2114A01C872FA0103008B5003108FC
:100EE000B60020160310A10D3508B7003608B8006B
:100EF0000327031C862F3508B7003608B800CD2617
:100F0000A40069260A128A11A400872F2114201137
:100F10002208031D9F2F0A30A200FF30A100B40158
:100F20003408A03E8400831380013408A83E840066
:100F300083138001B40A08303402031C902F210867
:100F40005926F0000330700203182015201DAB2F26
:100F5000A801A9014D2FA019201E4D2FA01120126C
:100F6000F8250A30A2004D2FF601F11FBE2FF0091F
:100F7000F00A0319F103F1097617F617730880399F
:100F8000F606F31FCA2FF209F20A0319F303F30955
:100F9000CA2FF601F401F501720873040319003435
:100FA0001F30F6040310F60AF20DF30D031CD32FC5
:100FB000F30CF20C73087102031DE02F720870022B
:100FC000031CE82F7208F0027308031C730AF10275
:100FD000F40DF50DF60BF61AD82FF61FF42FF409C1
:100FE000F40A0319F503F5097408F2007508F30013
:100FF000761F0034F009F00A0319F103F1090034F7
:02400E00723905
:00000001FF
